:105E6500011300001D0101010200000301FA0400F5
:105E7500FA0500030A0A5A0B001E0C00FA0D00036E
:105E85000E00030F0164100096120132130AFA1472
:105E9500010215000217010A1801FA1905321A0143
:105EA5000A1B01FA1C05321FFFFF20FFFF23011EFD
:105EB5002400642A00FA2B00FA2C50782D003D2E80
:105EC50000462F001E3000643250783432FA350116
:105ED50064360164370150380A643C00643E003C76
:105EE5003F000140FFFF411450420A5A430AC8448B
:105EF50005324500B44600FA4701484802034C0004
:105F0500FA4EFFFF500808510596520A32530B46C8
:105F1500540A96560000570546580002590A465A33
:105F250032FA5B010A5C0A325E000A5F00FE61FF1D
:105F3500FF6402116600026701016A0A3C6B0000FA
:105F45006C32967300007400007801327901327E5C
:105F5500FFFF81FFFF84FFFF8500AF8600018700FB
:105F6500FA89010A8A00009900009D0A969E00019F
:105F75009FFFFFFAFAFA0065006F00790083008D34
:105F8500009700A100AC00B600C000CA00D400DE36
:105F950000E800F2005B0063006A0072007A00828C
:105FA50000890091009900A100A800B000B800BFC9
:105FB50000C700CF00D600DF00E600EE00F6004087
:105FC5000046004C00520059005F0065006B0071EF
:105FD5000077007D00830089008F0095009C00A25A
:105FE50000A800AE00B400BA00C000C600CC00D2C4
:0A5FF50000D900DF00E500EB00F129
:1035E7009007BCE0FEA3E0FF905E67126138E493AA
:1035F700F599905E65E493FC740193FDEFB50507BB
:10360700EEB50403754D009007BC12611F2285F9C2
:103617007285FA737E017F00E573126111E5722FDF
:10362700FF50010E8E598F5A900013E0FCA3E0FD66
:10363700EF2DFDEE3CFC8C5B8D5C2275A71085F9A8
:103647007285FA737E017F00E573126111E5722FAF
:10365700FF50010E8E598F5A900013E0FCA3E0FD36
:10366700EF2DFDEE3CFC8C5B8D5C22E55CF5FBE50C
:103677005BF5FCD29322E55CF5E9E55BF5EAD294CC
:1036870022E55CF5EBE55BF5ECD29122E55CF5ED27
:10369700E55BF5EED29222E55CF5FBE55BF5FCD246
:1036A7008722E55CF5E9E55BF5EAD29022E55CF572
:1036B700EBE55BF5ECE5B54410F5B522E55CF5ED1A
:1036C700E55BF5EEE5B54420F5B522AE59AF5A7482
:1036D7000A8E048F05FF1261018C5B8D5CAE59AFBA
:1036E7005A740A8E048F05FF12612C8C598D5AE586
:1036F7005A45596013740AC3955AFFE49559FE8ECB
:10370700598F5A785B126165E55D2412F572E5728F
:10371700C3955CFFE4955BFE8E5B8F5C7424BE00F3
:10372700039F500974241261558E5B8F5CAE5BAFAB
:103737005C74246F4E700B755C23755B00757201AA
:1037470080037572002290008CE0B40104C21080DF
:1037570002D21090008DE0B40104C2118002D21190
:103767009000CAE075F0DCA4FFAEF0740A8E048FF7
:1037770005FF1261019007B2ECF0A3EDF0A20D4036
:103787001674038C068D07126111740112003990AB
:1037970007B0EEF0A3EFF07E017F00900088E01203
:1037A70061119000CBE08E048F05FF126101740A4E
:1037B700FF1261018D5F9000D4E075F0DCA4FFAECD
:1037C700F0740A8E048F05FF1261019007B6ECF0C2
:1037D700A3EDF09000D6E060139000D6E0F5F0740A
:1037E7001684FF7E00EF9007C0F080067464900790
:1037F700C0F09000CCE0900070F0900116E09000CF
:103807005AF09000A5E090005CF09000CEE09000A8
:103817005DF090007AE090005EF0900100E090008B
:1038270063F074E390006FF09000B5E0B40B087498
:10383700E390006FF0805A9000B5E0B41912900041
:10384700CBE0905F6612008CE49390006FF08041AC
:103857009000B5E0B41E129000CBE0905F84120098
:103867008CE49390006FF080289000B5E0B42812A4
:103877009000CBE0905FAE12008CE49390006FF065
:10388700800F9000B5E0B446089000ACE090006F60
:10389700F0900073E0FE9000B2E0B506339000743C
:1038A700E0FE9000DEE0B50627900075E0FE900090
:1038B700D0E0B5061B900077E0FE900085E0B506E6
:1038C7000F900076E0FE9000C0E06E7003023A555C
:1038D7009000C0E0640360069000DEE060087408B2
:1038E700900101F08006740A900101F09000C0E099
:1038F700B403089000DEE064026002800674009062
:1039070000DEF0900085E0B4010674009000EBF053
:10391700900085E0B4020674009000D0F090008516
:10392700E0B4030674009000DDF09000DEE0B4011F
:10393700147417900104F074009006C6F074009098
:1039470006C7F0800C7400900104F074179006C647
:10395700F09000D0E0D3940140147418900103F064
:1039670074009006CAF074009006CBF0800C7400C7
:10397700900103F074189006CAF09000B2E0B40208
:1039870014741990009AF074009006CEF0740090A9
:1039970006CFF0800C740090009AF074199006CE50
:1039A700F09000B2E06014741A900099F0740090DF
:1039B70006D2F074009006D3F0800C740090009942
:1039C700F0741A9006D2F09000C0E0B4020690009E
:1039D700DEE06002800E74079006DEF07408900641
:1039E700E2F0801874009006DEF074009006DFF0B5
:1039F70074009006E2F074009006E3F0D22890007D
:103A0700B2E0900073F09000DEE0900074F0900058
:103A1700D0E0900075F09000C0E0900076F0900044
:103A270085E0900077F0900085E090005BF09000D3
:103A3700C0E090005FF09000DEE0900060F0900042
:103A4700B2E0900061F09000D0E0900062F090004A
:103A5700E8E0B4011790001F740FF0A374FFF09013
:103A67000021E4F0A3F074029000E8F09000E8E091
:103A7700B40341900021E0FEA3E0FF90001FE0FCAB
:103A8700A3E0FD12615D7410126111740812003910
:103A9700EF90006CF0EF700674FF90006CF074000C
:103AA7009000E8F0900020E090006DF090001FE09B
:103AB70090006EF0900079E090003BF090003BE0C2
:103AC700240990003CF090003BE0241290003DF068
:103AD70090003BE0241B90003EF090003CE0D39424
:103AE70024400B90003CE0C3942490003CF09000ED
:103AF7003DE0D39424400B90003DE0C39424900014
:103B07003DF090003EE0D39424400B90003EE0C38C
:103B1700942490003EF0900079E0FE9000DCE02EC7
:103B2700900044F0900044E064126007900044E085
:103B3700B42406900044E004F0900044E0D39424B9
:103B4700400B900044E0C39424900044F09000445C
:103B5700E0D39412400D900044E0C39412900045C6
:103B6700F0800A900044E02412900045F07550124E
:103B77009000BFE090003FF090003FE075F00984AF
:103B8700AFF07E00EF4E700690003FE004F090002B
:103B97003FE0B4490690003F7401F090003FE0D346
:103BA7009424400F90003FE0C3942490003FF0D24C
:103BB700228002C22290003FE02409900040F0904A
:103BC700003FE02412900041F090003FE0241B905A
:103BD7000042F0900040E0D39424400B900040E076
:103BE700C39424900040F0900041E0D39424400B0C
:103BF700900041E0C39424900041F0900042E0D34C
:103C07009424400B900042E0C39424900042F02299
:103C1700C293C294C291C292C287C290E5B554EFD3
:103C2700F5B5E5B554DFF5B5C296C295C2A0C29702
:103C3700C2A2C2A1E5B554BFF5B5E5B5547FF5B548
:103C4700E5B554FBF5B5C212755D469000C2E0704C
:103C570005756C028003756C0375540075530090ED
:103C6700000874FFF0A374DCF0C219C21B74C8907B
:103C77000033F074C8900037F0755200755100C2D8
:103C87000D754600E56EB40903756E007562009008
:103C97000015E4F0A3F0756F10C215C216C217C263
:103CA700189007B2E0FEA3E0FF74031261117401DC
:103CB7001200399007B0EEF0A3EFF0C2027556007C
:103CC70075550090000CE4F0A3F0C22975580075F3
:103CD7005700900084E075F032A4FDACF090001D11
:103CE700ECF0A3EDF0C2392285F97285FA737E01F3
:103CF7007F00E573126111E5722FFF50010E8E5997
:103D07008F5AAC5BAD5CEF2DFDEE3CFC8C5B8D5CA4
:103D170012367212367D1236881236939000C0E042
:103D2700B4032C75A71085F97285FA737E017F009D
:103D3700E573126111E5722FFF50010E8E598F5AEC
:103D470012369E1236A91236B41236C375A7002250
:103D570075A71085F97285FA737E017F00E57312E6
:103D67006111E5722FFF50010E8E598F5A7E017F28
:103D7700769000FDE0126111AC59AD5AED2FFFECC2
:103D87003EFE8E5B8F5CE55CF5FDE55BF5FE900026
:103D970070E4F075A7007412900047F02285F9725D
:103DA70085FA737E017F00E573126111E5722FFFBB
:103DB70050010E8E598F5A9007B2E0FCA3E0FDEF39
:103DC7002DFDEE3CFC8C5B8D5CE55CF5FDE55BF564
:103DD700FE220563229000C0E0640360079000DEC6
:103DE700E0B4021EA2D8B34002C293A2D9B34002E4
:103DF700C294A2DAB34002C291A2DBB34002C292DC
:103E07008044A2D8B3400AC2939000DEE06002C2A9
:103E170087A2D9B3400AC2949000DEE06002C29044
:103E2700A2DAB3400EC2919000DEE06006E5B55419
:103E3700EFF5B5A2DBB3400EC2929000DEE060065C
:103E4700E5B554DFF5B5A2DCB34004C296C295755B
:103E5700D8402285A77175A7109000C0E064036061
:103E6700079000DEE0B40224A2D8B34002C287A2C2
:103E7700D9B34002C290A2DAB34006E5B554EFF5D4
:103E8700B5A2DBB34006E5B554DFF5B5A2DCB34018
:103E9700089000CCE0900070F075D8408571A7229B
:103EA700900047E4936406600280FE74C89007B8E8
:103EB700F8E4F0E8A3F075B50075840175A70075FF
:103EC700FFA0900043E4F075C91075A70F75A1C74F
:103ED70075A70075D90075CE0C75A70F75F1FE751E
:103EE700F2FF75F30775F47875A4BA75A5FF75A683
:103EF7000775AE0075AFFF75D48175D5FF75D6FF11
:103F070075D7FF75A70075A20175A14775F80975E3
:103F1700D80075D90475DA0975DB0975DC0975DD13
:103F27000975DE0975D84075A71075D80075D904CD
:103F370075DA0975DB0975DC0975DD0975DE097543
:103F4700D84075A70075E60875E71075BC0175BE02
:103F57000475BD6C75BE0775BDA075BE0875BD013E
:103F670075BC0075BB1875BC2075BA0875E88075F7
:103F7700D11375A70F75E10575E20075C740123CAF
:103F870017759700759780740A1260F17597C0E5E9
:103F9700975420700280F8758F0275A700D2AF750D
:103FA700980075A90C75A70F75AB4375ADFB75AC7C
:103FB7001E75A71075C91875CA0075CB0075C8049A
:103FC70075A700758912758E04758C00758A00C2F5
:103FD700A9D28C758D00758B00D2ABD28E75EF068A
:103FE70075D944C29974C8F5097508001200E375BC
:103FF700B5001204E374639007B8F8E4F0E8A3F09F
:1040070012036F74C89007B8F8E4F0E8A3F074647B
:10401700F5097508001200E390005BE0900085F059
:10402700C21F900085E0D39403400674009000857A
:10403700F0900085E0905A86F82828738028A2B46B
:104047004002D21F802075A70F75F30F75A700A236
:10405700A34002D21F800F75A70F75F31775A7002E
:06406700A2A44002D21FDA
:0C5A860002404302404502404D02405ED9
:10406D00A21FB34066757208E572D3940E5020E519
:10407D00729007B8F8E4F0E8A3F012023E7464F50C
:10408D00097508001200E37872740126F650D97490
:10409D00029000C1F0900085E0D3940340067400B7
:1040AD00900085F0900085E0905A92F82828738052
:1040BD001674009000EBF0800E74009000D0F0802C
:0740CD000674009000DDF015
:0C5A92000240BC0240BE0240C60240CEF2
:1040D400D21E8064757201E572D394075020E57294
:1040E4009007B8F8E4F0E8A3F012023E7464F5090E
:1040F4007508001200E37872740126F650D9740131
:104104009000C1F0900085E0D394034006740090C1
:104114000085F0900085E0905A9EF8282873801658
:1041240074009000EBF0800E74009000D0F08006D4
:0641340074009000DDF0B4
:0C5A9E0002412202412402412C0241344A
:10413A00C21E90005AE0900116F090005BE09000D9
:10414A0085F090005CE09000A5F090005DE09000A2
:10415A00CEF090005EE090007AF090005FE0900070
:10416A00C0F0900060E09000DEF0900061E0900006
:10417A00B2F0900062E09000D0F0900063E090010D
:10418A0000F09000CBE07006740A9000CBF090002B
:10419A00ACE0700674E39000ACF09000B2E00490DA
:1041AA000073F012374DE5B54401F5B57406900079
:1041BA0049F0740190004AF0740390004CF07405C1
:1041CA0090004DF0743C90004EF0740590004FF052
:1041DA007400900050F07400900055F07400900044
:1041EA0056F07401900057F07400900058F074FF74
:1041FA00900059F0743390014FF07436900150F0EA
:10420A00742D900151F07431900152F07420900194
:10421A0053F0744C900154F07465900155F0747821
:10422A00900156F07475900157F07473900158F02C
:10423A007432900159F0744390015AF0746F9001EE
:10424A005BF0746990015CF0746C90015DF0900011
:10425A00E7E090006CF090009EE090006DF0900016
:10426A009FE090006EF0A2B6B3920EA2B3B3920F83
:10427A00A2A4B39225A2B4B39226A2A3B392279082
:10428A000068E4F0756E00743A900778F074FD9057
:10429A000779F0900069E4F09007B2E0FEA3E0FF2E
:1042AA00740312611174011200399007B0EEF0A381
:1042BA00EFF0756D01900047E4F0C224756200C208
:1042CA0013D214C202757000C22BD203C22CD204BC
:1042DA00C22DD205C22ED206C22FD207C230D208B0
:1042EA00C231D209C232D20AC233D20BC234D20C80
:1042FA00C220C221C222C223C22812009E755E00B9
:10430A00756A0075600075643275650075660075BA
:10431A006700756800756900900015E4F0A3F075F0
:10432A006B00D2B2D2A4D2B0D2B1D2A3D2A7D2A6B3
:10433A00D2A5D2B7900084E0D394FA400674FA90DA
:10434A000084F07E017F0090006EE01261119000FF
:10435A006DE02FFF50010E90001FEEF0A3EFF0EF7B
:10436A00D394FFEE940F400790001FE4F0A3F0905F
:10437A00006CE0700674FF90006CF074009000AB63
:10438A00F09000C1E0D39402400674019000C1F09D
:10439A009000C2E07005756C028003756C03900092
:1043AA00C3E0D39401400674009000C3F09000C9A2
:1043BA00E0C3940A5006740A9000C9F09000D3E052
:1043CA00700674019000D3F09000D3E0B4FF067435
:1043DA00FE9000D3F09000DAE0D394FE400674FE1B
:1043EA009000DAF0900100E0D39402400674019044
:1043FA000100F0900116E0D3940140067401900187
:10440A0016F074019000E0F074019000E1F074007D
:10441A009000E8F07400900108F074299006BEF04C
:10442A00742A9006C2F0741B9006D6F0741C90068B
:10443A00DAF0D29C9000B3E0D3940440067404905E
:10444A0000B3F09000E5E0D39404400674049000B1
:10445A00E5F0E56FD394104003756F109006BFE046
:10446A00D3940C400674009006BFF09006C3E0D3C4
:10447A00940C400674009006C3F09006C7E0D394EB
:10448A000C400674009006C7F09006CBE0D3940C5B
:10449A00400674009006CBF09006CFE0D3940C400F
:1044AA000674009006CFF09006D3E0D3940C400631
:1044BA0074009006D3F09006D7E0D3940C400674AB
:1044CA00009006D7F09006DBE0D3940C4006740007
:1044DA009006DBF09006DFE0D3940C40067400905F
:1044EA0006DFF09006E3E0D3940C400674009006D1
:1044FA00E3F0D2EC75CF01A298B34005C298120638
:10450A0016E54D6006A299B3B340028005C299121E
:10451A000AB4E54E64016005E54EB4040280D5C2D2
:10452A008E7E107F00E563126111E58D75F010A48F
:10453A00FDACF0EF2DFDEE3CFCE58B75F01084FF31
:10454A007E00ED2FFFEC3EFE8E538F54D28E9000EC
:10455A00A5E060099000A5E0C3943D4002805C900C
:10456A00001712611F900017E0FEA3E0FF900019E8
:10457A00E0FCA3E0FDEFB50542EEB5043EB21DA294
:10458A000DB3401975E700A21DB34008E5B5440410
:10459A00F5B58006E5B554FBF5B575E71090001939
:1045AA00E0FEA3E0FF90001BE0FCA3E0FDEF2DFD81
:1045BA00EE3CFC900019ECF0A3EDF09000B2E06044
:1045CA00099000B2E0C394034002806F1229C0A28E
:1045DA000DB35009900068E0C394324002800690FF
:1045EA00009CE0F545E54575F005A4FFAEF090079F
:1045FA00BAEEF0A3EFF0900089E0C395604007E5BA
:10460A005EC3955F50079007BAE4F0A3F0AE2EAFF1
:10461A002F9007BAE0FCA3E0FDEFD39DEE9C400487
:10462A00C2A1800B900068E0C394445002D2A190CA
:10463A0000B2E0B40205A2A1B392A29000B2E0B423
:10464A00031C122ADBAE2EAF2F9007BAE0FCA3E0C0
:10465A00FDEFD39DEE9C4004D2A18002C2A190003E
:10466A008DE06009A2B3300F01B3B340028039A2D2
:10467A00B3300F01B34031A2B3301101B3401C90E3
:10468A0000C0E0B40306A220B3B34002800674045B
:10469A00900047F0D220A211B3920FA211B330B307
:1046AA0001B34004A211920FA2B6300E01B3500317
:1046BA00024D5DA2B6300E01B35003024D5DA2B6A3
:1046CA00301001B35003024B66756D009000A5E0EF
:1046DA00B43D1975E700A210B34008E5B554FBF5DF
:1046EA00B58006E5B54404F5B575E710055DA21277
:1046FA00B3B35013AE53AF54900008E0FCA3E0FDEF
:10470A00EDC39FEC9E400302485AE56CB4032EA207
:10471A0029B34022E55DB42403756C01E55DC394B9
:10472A002450069000477401F0E55DD394244006B6
:10473A007402900047F0755D01D229805AE56CB485
:10474A000206756C01755D24E55DB42405755D018D
:10475A008045900047E07030E55DC3942450069090
:10476A0000477401F0E55DD394244006740290007A
:10477A0047F0E55DC394245002D224E55DD3942426
:10478A004002D224C296C2959000C2E0B40105123A
:10479A003C178003755D01AE55AF56AC53AD54EF6F
:1047AA002DFDEE3CFC7403FF1261018C558D569071
:1047BA0000A5E060099000A5E0C3943D4002804353
:1047CA00900017E0FEA3E0FF9000A5E08E048F059D
:1047DA00FF12610174018C068D0712003990001BCB
:1047EA00EEF0A3EFF090001BE0F8A3E0900019C8E8
:1047FA00F0A3C8F0900017E4F0A3F0C21DE5B55489
:10480A00FBF5B5A2B4B34002C226A2A4B34002C2C9
:10481A0025A2A3B34002C227A224B34002C224A203
:10482A0020B34006A22292218002B22190008DE09C
:10483A006012E56C700EA220B35009A22130220149
:10484A00B3B3400280067405900047F0C220803A54
:10485A00AE55AF56AC53AD54EF2DFDEE3CFC740192
:10486A008C068D071200398E558F56E56CC394025B
:10487A00500DAC53AD547488C39D74139C40028090
:10488A0009123C177406900047F0E55DB4241274CF
:10489A0003900047F0D2249000C2E0B40103123C16
:1048AA0017AE57AF58AC53AD54EF2DFDEE3CFC8C10
:1048BA00578D58AE53AF54EFD39DEE9C40119000E4
:1048CA000FE0FAA3E0FBEBC394E8EA94034002800A
:1048DA000690000F12611F90000CE0FEA3E0FFACEF
:1048EA0053AD54EF2DFDEE3CFC90000CECF0A3ED23
:1048FA00F09000C2E0B4011DAE53AF5474051261CA
:10490A001174038E048F05FF126101900008ECF008
:10491A00A3EDF08016AE53AF547403126111740103
:10492A00120039900008EEF0A3EFF0C28E758D00E8
:10493A00758B00756300755401755300D28EE55D61
:10494A00240875F00984AFF07E00EF4E7075900070
:10495A000CE0F8A3E090000AC8F0A3C8F090000A9F
:10496A00E0FEA3E0FFEF4E600B7C807D0E125FFF3E
:10497A008E518F5290000CE4F0A3F0AE51AF5274F6
:10498A0028BE00039F5010E5622FFF50010E7401EC
:10499A001200398E518F528552629000C9E0A85197
:1049AA00B8000DD395524008E552900046F08009B0
:1049BA009000C9E014900046F0E56C60067552005C
:1049CA007551009000C0E0B4030890003FE0655DB7
:1049DA006002800BA221B34004D2238002B223E5F5
:1049EA005D640B6005E55DB41D099000B2E06003EB
:1049FA0012202B900044E0655D6007900045E0B509
:104A0A005D03756E00A213B35006A212B3B340033E
:104A1A00024AC290007EE0B40173900100E0B40241
:104A2A0014120C55900071E075F0BEA4FFAEF08E22
:104A3A005B8F5C8056E56675F00A84FF7E00900500
:104A4A0078126138E0F55A755900AE59AF5A90009C
:104A5A00A3E012611174648E048F05FF1261018C48
:104A6A005B8D5CE55C90000EF0AE59AF5A90007C0D
:104A7A00E012611174648E048F05FF12610174BE25
:104A8A008C068D071261118E5B8F5C801790007CFB
:104A9A00E075F0BEA4FFAEF08E5B8F5C9000A3E0E1
:104AAA0090000EF0E560C394CC500690007CE07054
:104ABA00028003123CEFD213E56CB40106E55D6493
:104ACA000B60028009756F019000487401F0E56C73
:104ADA006003024B619000C5E0600D900070E0A891
:104AEA0051B800069552400280489000C5E0B402D1
:104AFA002790003BE0655D601790003CE0655D60D3
:104B0A000F90003DE0655D600790003EE0B55D03F3
:104B1A00756F03756B00800CC200756B00900015F1
:104B2A00E4F0A3F0900070E060067409900047F08A
:104B3A008025E55D640A6005E55DB41C03756F01B7
:104B4A00A23A4010E55D64016005E55DB4130375A2
:104B5A006F0B8003756F03A210B3920EA210B330CD
:104B6A00B601B35003024D5D756D019000A5E0B426
:104B7A003D1975E700A210B34008E5B54404F5B540
:104B8A008006E5B554FBF5B575E710E5B54401F5C2
:104B9A00B57432900068F0A210920EE55DD3944A83
:104BAA004014D212E55DD3946E400B740490004712
:104BBA00F0D224755D469000CDE0B40107E569C3E3
:104BCA00941440028009123C177413900047F0A213
:104BDA002B300301B3501D75E700A22BB34008E543
:104BEA00B54408F5B58006E5B554F7F5B575E7108F
:104BFA00A22B9203A22C300401B3501D75E700A228
:104C0A002CB34008E5B54402F5B58006E5B554FD78
:104C1A00F5B575E710A22C9204A22D300501B35008
:104C2A000FA22DB34004D2A08002C2A0A22D9205E9
:104C3A00A22E300601B3500FA22EB34004D29780A1
:104C4A0002C297A22E9206A22F300701B3500FA2DA
:104C5A002FB34004D2A28002C2A2A22F9207A2308E
:104C6A00300801B3500FA230B34004D2A18002C26F
:104C7A00A1A2309208A231300901B3501D75E70094
:104C8A00A231B34008E5B54440F5B58006E5B55410
:104C9A00BFF5B575E710A2319209A232300A01B305
:104CAA00501D75E700A232B34008E5B54480F5B55A
:104CBA008006E5B5547FF5B575E710A232920AA2CF
:104CCA0033300B01B3501D75E700A233B34008E53A
:104CDA00B54410F5B58006E5B554EFF5B5A23392A3
:104CEA000B75E710A234300C01B3501D75E700A212
:104CFA0034B34008E5B54420F5B58006E5B554DF80
:104D0A00F5B5A234920C75E710E569C394415009D0
:104D1A00740E900047F0123C1790004FE0FE90008E
:104D2A004BE0C39E400990004BE0D39406400974BF
:104D3A00FB900047F0123C17900054E06015900079
:104D4A0054E0FE90004EE06E600974FE900047F059
:104D5A00123C17A224B34004C296C2959000FDE00B
:104D6A00600CAE51AF527414BE00059F40028048D9
:104D7A00900085E0905AAAF8282873803BA2B4B321
:104D8A005005A226B340028005123D57D22680283C
:104D9A00A2A3B35005A227B340028005123D57D201
:104DAA00278015A2A4B35005A225B340028005129C
:084DBA003D57D2258002800064
:105AAA00024D85024D87024D9A024DAD024DC0024C
:025ABA004DC2DB
:104DC200A215B3B3500890003FE0655D6003024E48
:104DD20087A201B35006A200B3B34003024E7F90F4
:104DE20000C0E0B4035EA20DB34030A223B340087A
:104DF200123615123672800912364212369E75A785
:104E0200009000DEE0B4011175E700A202B3400495
:104E1200D2A08002C2A075E7108027123615123682
:104E22007212364212369E75A7009000DEE0B4017F
:104E32001175E700A202B34004D2A08002C2A0759D
:104E4200E71080399000DEE0C39402500F1236154D
:104E5200123672A202B34002D28780211236151294
:104E62003672123642AE59AF5AAC2CAD2DEF2DFD33
:104E7200EE3CFC8C5B8D5C12369E75A700C215D28F
:104E820016D217D218A216B3B35008900040E065AC
:104E92005D6003024F4CA201B35006A200B3B340BF
:104EA20003024F449000C0E0B4035EA20DB3403051
:104EB200A223B3400812361512367D8009123642FB
:104EC2001236A975A7009000DEE0B4011175E70063
:104ED200A202B34004D2A08002C2A075E7108027CC
:104EE20012361512367D1236421236A975A7009077
:104EF20000DEE0B4011175E700A202B34004D2A0C3
:104F02008002C2A075E71080399000DEE0C39402EF
:104F1200500F12361512367DA202B34002D2908093
:104F22002112361512367D123642AE59AF5AAC2CCA
:104F3200AD2DEF2DFDEE3CFC8C5B8D5C1236A97520
:104F4200A700D215C216D217D218A217B3B35008AF
:104F5200900041E0655D6003025015A201B3500666
:104F6200A200B3B3400302500D9000C0E0B4035E50
:104F7200A20DB34030A223B3400812361512368870
:104F820080091236421236B475A7009000DEE0B4F2
:104F9200011175E700A202B34004D2A08002C2A0B0
:104FA20075E71080271236151236881236421236ED
:104FB200B475A7009000DEE0B4011175E700A2020B
:104FC200B34004D2A08002C2A075E710803D9000D9
:104FD200DEE0C394025013123615123688A202B3D1
:104FE2004006E5B54410F5B5802112361512368813
:104FF200123642AE59AF5AAC2CAD2DEF2DFDEE3C20
:10500200FC8C5B8D5C1236B475A700D215D216C229
:1050120017D218A218B3B35008900042E0655D6041
:10502200030250DEA201B35006A200B3B340030252
:1050320050D69000C0E0B4035EA20DB34030A2236C
:10504200B3400812361512369380091236421236D0
:10505200C375A7009000DEE0B4011175E700A2025B
:10506200B34004D2A08002C2A075E7108027123696
:10507200151236931236421236C375A7009000DE1F
:10508200E0B4011175E700A202B34004D2A080028D
:10509200C2A075E710803D9000DEE0C39402501379
:1050A200123615123693A202B34006E5B54420F536
:1050B200B58021123615123693123642AE59AF5AC6
:1050C200AC2CAD2DEF2DFDEE3CFC8C5B8D5C1236D5
:1050D200C375A700D215D216D217C218E56F905A1F
:0C50E200BCF82828730254999000E5E007
:065ABC000250E70250EA6F
:1050EE00905AEFF8282873121B078012121B0780A4
:0E50FE000D121B918008121C3D8003121C3DF8
:0F5AEF000250F50250FA0250FF02510402510911
:10510C00756F02025499121D69121E80A239B340A8
:10511C00229000A7E0F56B900078E0256BFE9000E4
:10512C0046E075F01E84FC7F00EE2CF53474109074
:10513C000047F09007B0E0FEA3E0FF740A12611183
:10514C0090000AE0FCA3E0FD74098F02FF126101DC
:10515C008D078C038E048A058B06125FFF9007B4B3
:10516C00EEF0A3EFF07478BE00039F500B747890B0
:10517C0007B4F8E4F0E8A3F0E5347003753401905B
:10518C0007B4E0FEA3E0FFE5342FFF50010E9007BB
:10519C00B4EEF0A3EFF0756F03A23A4003756F0AFB
:1051AC000254999006BFE060031221149000FEE0B7
:1051BC00B401149000FFE0A851B8000495525007B8
:1051CC00E55EC3955F400280030252599000B3E044
:1051DC00D39402403F900087E02403A851B8000408
:1051EC0095525009900089E0D3956050028008D206
:1051FC00017408900047F0900087E0A851B80005B2
:10520C00D39552500B900089E02403C39560500253
:10521C00C2018039900087E02403A851B80004959E
:10522C00525007E55EC3955F40028008D2017408B6
:10523C00900047F0900087E0A851B80005D3955234
:10524C005009E55F240FC3955E5002C2019000CD5A
:10525C00E07007E569C3941440028002D201A201F8
:10526C004005756F04800A756F10900015E4F0A36B
:10527C00F0A20DB34029E56675F00A84FF7E00901C
:10528C000578126138E0C394695005122060800FD4
:10529C009007B2E0F8A3E09007B0C8F0A3C8F00202
:0652AC0054999000B3E0EC
:095AC2000251120251AF0252AE72
:1052B200905AFEF8282873120D3F8012120D3F807B
:0E52C2000D120EED8008120F9F8003120F9F39
:0F5AFE000252B90252BE0252C30252C80252CD26
:1052D0009006C3E060031221F0756F050254991225
:1052E00010AB756F069006C7E060031222E09006CF
:1052F000CBE060031223BC02549990000EE06006DC
:10530000A20DB3B34002801D90000EE02529FFAE30
:105310002850010E8E288F29E55DD39412500690F7
:10532000000EE014F01212F1756F079006CFE060E6
:10533000031224989006D3E0600312257402549956
:10534000900100E0B40203120CCD12154E756F08E7
:105350009006D7E060031226509006DBE06003124F
:10536000272C02549912190AA215B35005A216B39C
:1053700040028008D215D216D217D218756F10903D
:1053800006DFE060031228089006E3E060031228BD
:10539000E4025499025499900035E0C394465008B1
:1053A000C2967446900035F085345A7559009000C5
:1053B0003BE0F5721236D2E55C900035F0900004C7
:1053C000E559F0A3E55AF0E572900036F0C21A9064
:1053D00007B4E0F559A3E0F55A90003BE0F57212EE
:1053E00036D2E55C900033F0900000E559F0A3E57B
:1053F0005AF0E572900034F0C219E56CB4010575FD
:105400006F0B8003756F03025499900039E0C394C9
:105410004650139000CEE0B40104C2968002C295BB
:105420007446900039F085345A75590090003CE07C
:10543000F5721236D2E55C900039F0900006E5591D
:10544000F0A3E55AF0E57290003AF0C21C9007B460
:10545000E0F559A3E0F55A90003CE0F5721236D21F
:10546000E55C900037F0900002E559F0A3E55AF0B2
:10547000E572900038F0C21BE56CB4010F756C004A
:1054800074C8900033F074C8900037F0756F1080C6
:09549000088006800480028000FF
:105ACB000252DF0252FA0253400253650253940210
:105ADB00539702540A025491025493025495025460
:045AEB009702549931
:10549900900033E0B55D73A219404F900000E0FE23
:1054A900A3E0FFEF4E6021AE55AF56900000E0FC3F
:1054B900A3E0FD120003740A8E048F05FF12610137
:1054C900900000ECF0A3EDF0900034E0601A900039
:1054D90000E0FEA3E0FFAC55AD56EF2DFDEE3CFC20
:1054E900900000ECF0A3EDF0D219AE53AF54900048
:1054F90000E0FCA3E0FDEFC39DEE9C400D123DA42E
:10550900D296C21974C8900033F0A219B3B35007E8
:10551900900033E0B55D02800D123DA4D29674C8A7
:10552900900033F0C219900035E0B55D70A21A40C1
:105539004F900004E0FEA3E0FFEF4E6021AE55AFAF
:1055490056900004E0FCA3E0FD120003740A8E04E7
:105559008F05FF126101900004ECF0A3EDF09000BB
:1055690036E0601A900004E0FEA3E0FFAC55AD56AA
:10557900EF2DFDEE3CFC900004ECF0A3EDF0D21A07
:10558900AE53AF54900004E0FCA3E0FDEFC39DEEE1
:105599009C400AC2967446900035F0C21AA21AB30A
:1055A900B35007900035E0B55D02800AC296744693
:1055B900900035F0C21A900037E0B55D73A21B4028
:1055C9004F900002E0FEA3E0FFEF4E6021AE55AF21
:1055D90056900002E0FCA3E0FD120003740A8E0459
:1055E9008F05FF126101900002ECF0A3EDF090002D
:1055F90038E0601A900002E0FEA3E0FFAC55AD561A
:10560900EF2DFDEE3CFC900002ECF0A3EDF0D21B77
:10561900AE53AF54900002E0FCA3E0FDEFC39DEE52
:105629009C400D123DA4D295C21B74C8900037F05E
:10563900A21BB3B35007900037E0B55D02800D128D
:105649003DA4D29574C8900037F0C21B900039E090
:10565900B55D70A21C404F900006E0FEA3E0FFEF8D
:105669004E6021AE55AF56900006E0FCA3E0FD1256
:105679000003740A8E048F05FF126101900006EC85
:10568900F0A3EDF090003AE0601A900006E0FEA366
:10569900E0FFAC55AD56EF2DFDEE3CFC900006EC5D
:1056A900F0A3EDF0D21CAE53AF54900006E0FCA37A
:1056B900E0FDEFC39DEE9C400AC295744690003907
:1056C900F0C21CA21CB3B35007900039E0B55D02CB
:1056D900800AC2957446900039F0C21C9000D0E04F
:1056E900B40202800302580190006AE0D395655024
:1056F9006490006AE0F4042565FE9000D3E08E0012
:10570900F5F0E884FF7E008F72EFC39410500CEF20
:105719008572F0A4FDACF08D7280037572FF900064
:105729006AE0D39572400B90006AE0C39572F570F8
:1057390080037570009000EEE0D3957040069000EC
:10574900EEE0F5709000EFE0C3957050069000EF21
:10575900E0F570807190006AE0C39565FE9000D312
:10576900E08E00F5F0E884FF7E008F72EFC394109D
:10577900500CEF8572F0A4FDACF08D728003757248
:10578900FF85725A75590090006AE0255AFFAE5993
:1057990050010E8E598F5A74FFBE0009D39F4005E0
:1057A900855A7080037570FF9000EEE0D3957040C4
:1057B900069000EEE0F5709000EFE0C3957050069A
:1057C9009000EFE0F570A20DB3B3500D90006BE0BF
:1057D900FE9000DBE0D39E5002800A7407900047D8
:1057E900F0C297801375A710E5CDC395704004C228
:1057F900978002D29775A700E56EC39409500AA253
:10580900EDB34005C2ED122C7AAE53AF547410C3F8
:105819009F74279E400C900069E0C3945A4003028C
:105829005A83A212B34009123C177406900047F03C
:10583900A21FB34008E5B54404F5B58006E5B554A3
:10584900FBF5B5A214B3500EE560D394334007E5D8
:1058590060C394CC4002802FE5B54401F5B574329C
:10586900900068F090007CE075F0BEA4FFAEF08E69
:105879005B8F5C7402BE000AD39F4006755C02759B
:105889005B00123CEFD214900069E0D39401400709
:10589900E560C3941A40028002C2149006BFE0601A
:1058A90003122114A22B300301B35017A22BB340CA
:1058B90008E5B54408F5B58006E5B554F7F5B5A290
:1058C9002B92039006C3E060031221F0A22C30044E
:1058D90001B35017A22CB34008E5B54402F5B580D1
:1058E90006E5B554FDF5B5A22C92049006C7E06013
:1058F900031222E0A22D300501B3500FA22DB340AF
:1059090004D2A08002C2A0A22D92059006CBE0602D
:10591900031223BCA22E300601B3500FA22EB340AE
:1059290004D2978002C297A22E92069006CFE06019
:1059390003122498A22F300701B3500FA22FB340AE
:1059490004D2A28002C2A2A22F92079006D3E060DD
:1059590003122574A230300801B3500FA230B340AE
:1059690004D2A18002C2A1A23092089006D7E060B9
:1059790003122650A231300901B35017A231B340A6
:1059890008E5B54440F5B58006E5B554BFF5B5A2BF
:105999003192099006DBE0600312272CA232300A0B
:1059A90001B35017A232B34008E5B54480F5B5807C
:1059B90006E5B5547FF5B5A232920A9006DFE0609C
:1059C90003122808A233300B01B35017A233B34096
:1059D90008E5B54410F5B58006E5B554EFF5B5A26F
:1059E90033920B9006E3E060031228E4A234300CF2
:1059F90001B35017A234B34008E5B54420F5B5808A
:105A090006E5B554DFF5B5A234920C900069E0C300
:105A1900945A5010E56EB40909900069E004F075D4
:105A29006E00803BE56EB40903756E007554007510
:105A39005300758D00758B00756300900068E0C395
:105A490094445008900068E004F080067444900083
:105A590068F0900068E0B44406E5B554FEF5B590E9
:105A69000069E0D394014007E569C394414002808D
:0D5A790009740E900047F0123C170244FE25
:105B0D000000010001400160018001A001C001E021
:105B1D0002000300039603B603D603F40400050048
:105B2D000512052405360548055A056C057E0590B8
:105B3D0005A805C005DE0600061406280646066EF5
:105B4D0006AE00FF013F015F017F019F01BF01DF35
:105B5D0001FF02FF039503B503D503F303FF04FF14
:105B6D0005110523053505470559056B057D058F80
:105B7D0005A705BF05DD05F1061306270645066DCC
:105B8D0006AD06ED0FAA0FA50F9F0F9A0F940F8D5F
:105B9D000F870F800F780F710F680F600F570F4E23
:105BAD000F450F3B0F300F250F1A0F0E0F020EF57D
:105BBD000EE80EDB0ECC0EBE0EAE0E9F0E8E0E7DC3
:105BCD000E6C0E5A0E470E340E200E0C0DF70DE214
:105BDD000DCB0DB50D9D0D850D6D0D540D3A0D2093
:105BED000D050CE90CCE0CB10C940C760C580C3A3E
:105BFD000C1B0BFB0BDB0BBB0B9A0B790B570B35F4
:105C0D000B130AF10ACE0AAB0A870A640A400A1C72
:105C1D0009F809D409B0098C09670943091F08FB64
:105C2D0008D608B2088E086A0846082307FF07DC65
:105C3D0007B9079607730751072F070D06EC06CA1C
:105C4D0006AA068906690649062A060A05EC05CD47
:105C5D0005B0059205750558053C0520050504EAB6
:105C6D0004CF04B5049C0482046904510439042250
:105C7D00040B03F403DE03C803B2039D038903750C
:105C8D000361034D033B03280316030402F202E1F3
:105C9D0002D102C002B002A002910282027302651B
:105CAD0002570249023C022F02220216020901FD8F
:105CBD0001F201E601DB01D001C601BB01B101A773
:105CCD00019D0194018B01820179017001680160D0
:105CDD00015801500148014101390132012B0125C3
:105CED00011E01180111010B010500FF00FA0FA69D
:105CFD000FA00F990F920F8B0F840F7C0F740F6BEA
:105D0D000F620F580F4E0F430F380F2C0F1F0F122E
:105D1D000F050EF70EE80ED80EC80EB70EA50E9392
:105D2D000E800E6C0E580E420E2C0E150DFD0DE450
:105D3D000DCB0DB10D950D790D5D0D3F0D200D01A7
:105D4D000CE10CC00C9E0C7C0C590C350C100BEAA4
:105D5D000BC40B9E0B760B4F0B260AFD0AD40AAA19
:105D6D000A800A550A2A09FF09D409A8097C095095
:105D7D00092508F908CD08A10875084A081E07F37A
:105D8D0007C8079D07730749072006F706CE06A625
:105D9D00067E06570630060A05E405BF059B057706
:105DAD0005540532051004EF04CE04AE048F0471C2
:105DBD0004530435041903FD03E203C703AD039433
:105DCD00037B0363034B0334031E030802F302DE5C
:105DDD0002CA02B602A30291027F026D025C024C5E
:105DED00023C022C021D020E020001F201E401D759
:105DFD0001CA01BE01B101A6019A018F0185017A87
:105E0D0001700166015D0153014A01410139013102
:105E1D000129012101190112010B010400FD00F7F7
:105E2D0000F000EA00E400DE00D900D300CE00C986
:105E3D0000C400BF00BA00B500B100AD00A800A4B9
:105E4D0000A0009C009900950091008E008A0087AB
:085E5D0000840081007E007B3F
:10009E007547009007BCE4F0A3F075310075300091
:1000AE00754D00754E00C236D23774FE9007C6F8F5
:1000BE00E4F0E8A3F074FE9007C8F8E4F0E8A3F0CB
:1000CE00745A9007CAF0745A9007CBF0D238C22AED
:1000DE00C23AC23522750B00750A00AE0AAF0BACE0
:1000EE0008AD09EDC39FEC9E401674FF1260F175CA
:1000FE00CF01780B740126F6500418E436F650DB67
:10010E0022900043E0B4AA1C900778E0B43C15900E
:10011E0007B8E0FEA3E0FFEF4E6009741EBE0004B8
:10012E00D39F500302023D755C00755B0075F809A4
:10013E009007B8E0FEA3E0FF74076F4E6006740EE2
:10014E006F4E7006743A900778F09007B8E0FEA3F1
:10015E00E0FF7408BE001ED39F401A7E017F0890F8
:10016E0007B8E0FCA3E0FD1DBDFF011C1200038ECD
:10017E00598F5A801F9007B8E0FEA3E0FF74081253
:10018E0061558F048E057E017F08CDCCCD12000304
:10019E008E598F5AAE5BAF5C740CD39F74019E5018
:1001AE0003020238A2F9B3407EE55C455B7003752D
:1001BE00A382AE5BAF5C74016F4E700375A300AE8D
:1001CE005BAF5C74026F4E700D9007B9E075F00274
:1001DE00A4FDACF08DA3AE5BAF5C74036F4E7003E9
:1001EE0075A300AE5BAF5C7403BE00039F5013ACEF
:1001FE0059AD5AED2FFFEC3EFE900074126138E0BF
:10020E00F5A3AE5BAF5CEFB40B09EEB4010574144D
:10021E001260F1AE5BAF5CEFB40B07EEB401037589
:10022E00F80D785B1261650201A2900043E4F022A2
:10023E00755C00755B0075F8099007B8E0FEA3E0E9
:10024E00FF7408BE001ED39F401A7E017F089007E0
:10025E00B8E0FCA3E0FD1DBDFF011C1200038E598A
:10026E008F5A801F9007B8E0FEA3E0FF740812615A
:10027E00558F048E057E017F08CDCCCD1200038EE6
:10028E00598F5AAE5BAF5C7411D39F74019E5003AD
:10029E0002036EA2F9B3500302036BE55C455B707B
:1002AE000375A3D2AE5BAF5C74016F4E700375A382
:1002BE0000AE5BAF5C74026F4E700D9007B9E075C7
:1002CE00F002A4FDACF08DA3AE5BAF5C74036F4E79
:1002DE00700375A300AE5BAF5C74046F4E70037554
:1002EE00A300AE5BAF5C74056F4E700375A300AEDA
:1002FE005BAF5C74066F4E700375A300AE5BAF5CB4
:10030E0074076F4E700375A300AE5BAF5C74086F1D
:10031E004E700375A300AE5BAF5C7408BE00039F06
:10032E005016AC59AD5AED2FFFEC3EFE90006F12F9
:10033E006138E5A3F075A300AE5BAF5CEFB41009B6
:10034E00EEB4010574141260F1AE5BAF5CEFB41045
:10035E0007EEB4010375F80D785B12616502029128
:10036E0022755C00755B0075F809AE5BAF5C7417A7
:10037E00BE0004D39F5003020447A2F9B3500302F8
:10038E000444E55C455B700375A3D2AE5BAF5C7451
:10039E00016F4E700375A300AE5BAF5C74026F4EBF
:1003AE00700D9007B9E075F002A4FDACF08DA3AE10
:1003BE005BAF5C74036F4E700375A300AE5BAF5CF6
:1003CE0074046F4E700375A300AE5BAF5C74056F63
:1003DE004E700375A300AE5BAF5C74066F4E700378
:1003EE0075A300AE5BAF5C74076F4E700375A30010
:1003FE00AE5BAF5C74086F4E700375A300AE5BAF5F
:10040E005C7408BE00039F500C900051126138E5D9
:10041E00A3F075A300AE5BAF5C74166F4E700574DF
:10042E00141260F1AE5BAF5C74166F4E700375F80C
:10043E000D785B12616502037822900043E0B4AB45
:10044E000280030204E2755C00755B0075F809AE6C
:10045E005BAF5C7412BE007CD39F4078A2F9B340B0
:10046E0070E55C455B700375A382AE5BAF5C740197
:10047E006F4E700375A300AE5BAF5C74026F4E706F
:10048E000D9007B9E075F002A4FDACF08DA3AE5B44
:10049E00AF5C74036F4E700375A300AE5BAF5C74FC
:1004AE0003BE00039F5009900056126138E0F5A379
:1004BE00AE5BAF5C74116F4E700574141260F1AECA
:1004CE005BAF5C74116F4E700375F80D785B126143
:1004DE006502045D229007C3E4F074649007B8F8D7
:1004EE00E4F0E8A3F012036F74C89007B8F8E4F0D4
:1004FE00E8A3F090005DE0B4371A90005AE0900047
:10050E0051F090005BE0900052F090005CE09000A3
:10051E0053F080469007C37401F074659007B8F8E5
:10052E00E4F0E8A3F012036F74C89007B8F8E4F093
:10053E00E8A3F090005DE0B4371A90005AE0900006
:10054E0051F090005BE0900052F090005CE0900063
:10055E0053F0800674029007C3F09007C4E4F07461
:10056E00669007B8F8E4F0E8A3F012036F74C89031
:10057E0007B8F8E4F0E8A3F090005CE0B43712900E
:10058E00005AE090004BF090005BE0900054F08039
:10059E00769007C47401F074679007B8F8E4F0E839
:1005AE00A3F012036F74C89007B8F8E4F0E8A3F054
:1005BE0090005CE0B4371290005AE090004BF0903F
:1005CE00005BE0900054F0803E74029007C4F0741B
:1005DE00689007B8F8E4F0E8A3F012036F74C890BF
:1005EE0007B8F8E4F0E8A3F090005CE0B43712909E
:1005FE00005AE090004BF090005BE0900054F080C9
:10060E000674039007C4F022E54E64046006E59973
:10061E0064FF6002802AA2364004D2368020E54E66
:10062E00600874E6254E900047F0754E00E54D606B
:10063E000874F0254D900047F0754D00C2368002CB
:10064E00C236E54E9033F8F8282873754E00E599BA
:10065E00B4FF03754D01E599B4FE03754D02E5999E
:10066E00B4FD03754D03E599B4FC03754D04E5998E
:10067E00B4FA03754D05E599B4FB06754E01123CAF
:10068E0017E599B4F906754E04123C17E599D39403
:10069E00E54007E599C394F04002801685994F75A1
:1006AE004E027E017F00E54FC394E61261118E3239
:1006BE008F339007BCE4F0A3F0E599D394C44007C0
:1006CE00E599C394E64002802885994F754E0374D0
:1006DE00E5C3954FF533753200AE32AF33905B0DF7
:1006EE001260E0E493F87401939007BCC8F0A3C8BD
:1006FE00F0D299020AB390005AE070429007BCE023
:10070E00FEA3E0FF74FFBE00039F5009EFC39446A3
:10071E00EE940640119007BCE0FEA3E0FFEFD394E9
:10072E006DEE940640139007BCE0FEA3E0FF900030
:10073E0078126138E599F0800385997380119007DE
:10074E00BCE0FEA3E0FF900078126138E599F090CE
:10075E0007BC12611F9007BCE0FEA3E0FFEFB401DF
:10076E0006EEB40702800302089B900778E0B43CC3
:10077E00028003020885C29C90005AE0900116F098
:10078E0090005BE0900085F090005CE09000A5F09A
:10079E0090005DE09000CEF090005EE090007AF068
:1007AE0090005FE09000C0F0900060E09000DEF0FE
:1007BE00900061E09000B2F0900062E09000D0F006
:1007CE00900063E0900100F012374D90006CE090C5
:1007DE0000E7F090006DE090009EF090006EE090CB
:1007EE00009FF074639007B8F8E4F0E8A3F074ABE0
:1007FE00900043F0120448900043E4F075096475CC
:10080E0008001200E3A21E4038757201E572D394FF
:10081E0007502CE5729007B8F8E4F0E8A3F074AA3C
:10082E00900043F012010FE572C394075009750949
:10083E00647508001200E37872740126F650CD80BC
:10084E0036757208E572D3940E502CE5729007B887
:10085E00F8E4F0E8A3F074AA900043F012010FE55B
:10086E0072C3940E50097509647508001200E3787E
:10087E0072740126F650CD74C89007B8F8E4F0E80B
:10088E00A3F0D29C754E00754D007599FB020AB30C
:10089E009007BCE0FEA3E0FFEF4E70068599317520
:1008AE0030009007BCE0FEA3E0FF74016F4E701B9A
:1008BE00AC30AD31AA32AB33ED2BFBEC3AFA8A06F3
:1008CE008B07900078126138E599F09007BC1261A1
:1008DE001F9007BCE0FEA3E0FF74026F4E7021ACC8
:1008EE0030AD3174566D4C7006E54F64E660028093
:1008FE0003123C1712374D854F99754E00754D00FA
:10090E00020AB39007BCE0FEA3E0FF9000781261EC
:10091E0038E599F09007BC12611F9007BCE0FEA36A
:10092E00E0FFAC32AD338F028E038C068D07905BE9
:10093E004F1260E0E493F9740193FEEAD39EEB99B3
:10094E004009854F99754E00754D00020AB3900708
:10095E00BCE0FEA3E0FF900078126138E599F090BC
:10096E0007BC12611F9007BCE0FEA3E0FFEFB400CE
:10097E0006EEB401028003020AB3900053E075F054
:10098E0002A4FDACF08D72ED900078126143EDFA89
:10099E00E0FBEA90007B126143EBFAE0FBEA2BFAF4
:1009AE00900053E0B502028003020AA50DED9000FF
:1009BE0078126143E572FDE0FAED90007C1261431E
:1009CE00EAFDE0FAEDC39AFD900053E0B505028012
:1009DE0003020AA5E57290007A126143E572FDE00A
:1009EE00FAED90007D126143EAFDE0FAED2AFD90EA
:1009FE000053E0B505028003020AA5E57290007E61
:100A0E00126143FDE0FAED900053E0F4042A9000E9
:100A1E005AF0E57290007F126143FDE0FAED90000E
:100A2E0053E0F4042A90005BF0E5729000801261AE
:100A3E0043FDE0FAED900053E0F4042A90005CF0E0
:100A4E00E572900081126143FDE0FAED900053E0F3
:100A5E00F4042A9007B8F8E4F0E8A3F074AB900021
:100A6E0043F01204487509647508001200E39007FC
:100A7E00B812611F1204487509647508001200E36C
:100A8E009007B812611F1204487599F975096475BB
:100A9E0008001200E380FE7599FF75096475080061
:050AAE001200E380FED0
:0F33F80002065902070402089E02091102095C2D
:100AB30022E54D903407F8282873020B989007BC61
:100AC300E0FEA3E0FF900049126138E0F59990073A
:100AD300BC12611F9007BCE0FEA3E0FF74116F4ED0
:100AE3007003754D00020B98856D99020B98900762
:100AF300BCE0FEA3E0FF900078126138E0F599EFC7
:100B0300B40107EEB40703754D009007BC12611FD3
:070B1300020B989007BDE002
:0F340700020ABD020AC0020AEB020AF1020B160A
:100B1A009035BAF82828738552998067855E99803E
:100B2A0062856099805D856499805885669980534D
:100B3A00856799804E85689980498569998044902E
:100B4A000016E0F599803CA237B340077599FAC2BE
:100B5A00378017A228B3400575990F800B9000477C
:100B6A00E0F599900047E4F0C2288017856A9980D9
:100B7A0012856599800D856B9980087599FC8003AB
:030B8A00754D00A6
:1035BA00020B21020B26020B2B020B30020B3502E7
:1035CA000B3A020B3F020B44020B49020B51020B4E
:0D35DA0076020B7B020B80020B85020B8A30
:0B0B8D009007BC12611F80031235E7C7
:03341600020B9511
:100B980022E537255AFFAE5950010E9000781261B0
:100BA80038E0F538E537255AFFAE5950010E0FBF2A
:100BB80000010E900078126138E0F539853F3BE579
:100BC80038B539058538378041E539D39538401D22
:100BD800E539C39538853AF0A4FFAEF0E53B8E04BD
:100BE8008F05FF126101ED2538F537801DE538C303
:100BF8009539853AF0A4FFAEF0E53B8E048F05FFEA
:100C0800126101EDF4042538F53722E539D395381A
:100C1800401DE539C39538853AF0A4FFAEF0E53BB1
:100C28008E048F05FF126101ED2538F537801DE52B
:100C380038C39539853AF0A4FFAEF0E53B8E048FB2
:100C480005FF126101EDF4042538F5372290007E86
:100C5800E0B40170E56675F00A84FF7E008F37E521
:100C68006675F00A84ADF07C008D3A753F0A7559B7
:100C780005755A24E537C394115005120B9980065F
:100C88009005ADE0F537E537900071F0E56675F051
:100C98000A84FF7E008F37E56675F00A84ADF07C24
:100CA800008D3A753F0A755905755A5AE537C39448
:100CB800115005120B9980069005E3E0F537E537EA
:100CC80090000EF02290007EE0B4016AE56675F0AF
:100CD8000A84FF7E008F37E56675F00A84ADF07CE4
:100CE800008D3A753F0A755905755A36E537C3942C
:100CF800115005120B9980069005BFE0F53785372E
:100D08004BE56675F00A84FF7E008F37E56675F05F
:100D18000A84ADF07C008D3A753F0A755905755AFD
:100D280048E537C394115005120B9980069005D1F8
:100D3800E0F53785374C22E55E75F00484FF7E00C8
:100D48008F37E55E75F00484ADF07C008D3A753F11
:100D580004755901755A00E537C3943F5005120BC5
:100D68009980069001B7E0F53785372975280090F6
:100D78000046E075F020A4FFAEF09000C9E08E04B4
:100D88008F05FF1261018D379000B1E0D3955E5059
:100D980003020E459000D5E0D3955E4010ED90011A
:100DA800B8126143E0F52B752A00020E429000A0AC
:100DB800E0D3955E4043E5379001B8126143E0F512
:100DC80038E5379001D8126143E0F5399000D5E055
:100DD800F404255EF53A9000A0E0FE9000D5E0F41A
:100DE800042EF53BE538B539058538378003120CF4
:100DF8001385372B752A008041E5379001D8126199
:100E080043E0F538E5379001F8126143E0F5399091
:100E180000A0E0F404255EF53A9000B1E0FE9000F1
:100E2800A0E0F4042EF53BE538B539058538378060
:100E380003120C1385372B752A00020EEC9000D88C
:100E4800E0D3955E5011E537900238126143E0F522
:100E58002B752A00020EEC9000A1E0D3955E50435A
:100E6800E537900218126143E0F538E5379002380B
:100E7800126143E0F5399000A1E0F404255EF53AEB
:100E88009000D8E0FE9000A1E0F4042EF53BE53890
:100E9800B539058538378003120C1385372B752A29
:100EA800008041E5379001F8126143E0F538E537F5
:100EB800900218126143E0F5399000B1E0F404257E
:100EC8005EF53A9000A1E0FE9000B1E0F4042EF542
:100ED8003BE538B539058538378003120C1385375B
:100EE8002B752A00229000E9E0F53C753F117559F1
:100EF80002755A00AE51AF52E53C75F00FA4FDAC37
:100F0800F0EDD39FEC9E4021E53C8E048F05FF1247
:100F18006101ED75F010A4FFAEF0E55E75F0118487
:100F2800FD7C00ED2FF53D800EE55E75F01184FF28
:100F38007E00EF24F0F53D853D37E55E75F01184C0
:100F4800AFF07E008F3A120B9985373EAE51AF5203
:100F58009000E9E075F00FA4FDACF0EDD39FEC9E96
:100F68004028755902755A10853D37120B99853EF0
:100F780038853739AE51AF52E53C8E048F05FF12E4
:100F8800612C8D3A853C3B120C1385372975280056
:100F9800752B64752A00229000E9E0F53C753F1135
:100FA800755902755A00AE51AF52E53C75F00FA461
:100FB800FDACF0EDD39FEC9E4021E53C8E048F05FF
:100FC800FF126101ED75F010A4FFAEF0E56075F059
:100FD8001184FD7C00ED2FF53D800EE56075F01164
:100FE80084FF7E00EF24F0F53D853D37E56075F020
:100FF8001184AFF07E008F3A120B9985373EAE51BF
:10100800AF529000E9E075F00FA4FDACF0EDD39F6E
:10101800EC9E4028755902755A10853D37120B9978
:10102800853E38853739AE51AF52E53C8E048F0581
:10103800FF12612C8D3A853C3B120C1385372975BC
:1010480028009000B3E0B40453E55E75F00484FF13
:101058007E008F37E55E75F00484ADF07C008D3A34
:10106800753F04755901755A00E537C3943F50051B
:10107800120B9980069001B7E0F537AE28AF29E545
:101088003712611174648E048F05FF126101AE2856
:10109800AF29EF2DFDEE3CFC8C288D29752B64754E
:1010A8002A002290007EE0B40146E56675F00A84C5
:1010B800FF7E008F37E56675F00A84ADF07C008D01
:1010C8003A753F0A755905755A00E537C3941150AA
:1010D80005120B998006900589E0F537AE2AAF2BEB
:1010E800E5372FFF50010E74641261558E2A8F2B3D
:1010F80090007FE0B40146E56775F00A84FF7E0042
:101108008F37E56775F00A84ADF07C008D3A753F3E
:101118000A755905755A6CE537C394115005120BB9
:101128009980069005F5E0F537AE2AAF2BE5372F05
:10113800FF50010E74641261558E2A8F2B90008E19
:10114800E0B40249E569C3944175F00584FF7E0067
:101158008F37E56975F00584ADF07C008D3A753FF1
:1011680005755906755A00E537C394135005120BD7
:1011780099800690068BE0F537AE2AAF2BE5372F1E
:10118800FF50010E74641261558E2A8F2B9000D087
:10119800E0B40202800302124AE55E75F01584FF8E
:1011A8007E008F37E55E75F01584ADF07C008D3AD2
:1011B800753F15755903755AF4E537C3940B5005F7
:1011C800120B998006900477E0F537E53775F0FF44
:1011D800A4FFAEF09000D1E08E048F05FF126101EC
:1011E800ED90006AF0E56575F078A4FFAEF074FF45
:1011F8008E048F05FF1261018C598D5A74028C067A
:101208008D071200398F37AC59AD5A7404FF12613B
:101218002C8D3A753F04755906755A28E537C394DD
:101228001D5005120B9980069006BDE0F537AE2AD1
:10123800AF2BE5372FFF50010E74641261558E2ACB
:101248008F2B90007DE0B4025DE56075F064A4FF2B
:10125800AEF074081200398E5B8F5C74058E048FB3
:1012680005FF1261018D37AE5BAF5C74058E048F8C
:1012780005FF12612C8D3A753F05755905755ADEC3
:10128800E537C394135005120B998006900669E060
:10129800F537AE2AAF2BE5372FFF50010E746412D5
:1012A80061558E2A8F2B9000BFE0703C900046E07D
:1012B80075F00584FF7E008F37900046E075F005D5
:1012C80084ADF07C008D3A753F05755905755AC097
:1012D800E537C3941D5005120B998006900655E01A
:1012E800F537E537900072F022900086E0B40117D8
:1012F8009007BFE0252BFFAE2A50010E9000DAE0E0
:101308001261558E2A8F2B9000FEE0B401149000D4
:10131800FFE0A851B8000495525007E55EC3955FF9
:10132800400280129000A8E0252BFFAE2A50010E43
:101338008E2A8F2B802F900086E0B40316A22AB342
:10134800B350109007C2E0C39405A851B8000695A1
:1013580052400280109000A8E0252BFFAE2A5001D1
:101368000E8E2A8F2B900080E0B4020280030215B3
:101378004D900083E0602FE566D3944640289000A6
:101388000FE0FEA3E0FF9000BEE075F003A4FDAC03
:10139800F0EFD39DEE9C400E9000E2E0A851B8001B
:1013A80005D39552500302154D9000CBE0855EF0B1
:1013B800A4FFAEF0740512611174071200398E593A
:1013C8008F5A90008AE0A851B800049552501290A4
:1013D800008BE075F002A4FDACF0EFC39DEE9C40DD
:1013E8000302154DE55E75F00B84FF7E009006083C
:1013F800126138FEE0FFEE900082E0FEEF8E00887A
:10140800F0A4FFAEF074648E048F05FF1261018CA6
:10141800598D5A900046E075F018A4FFAEF0900080
:10142800C9E08E048F05FF1261018C068D079006B6
:1014380020126138AE59AF5AE012611174648E04FB
:101448008F05FF1261018C598D5AE564A859B800BF
:1014580077D3955A4072E564C3955AFFE49559FECF
:101468008E598F5A7428BE00039F500C755A2875E0
:101478005900740D900047F0AE59AF5A900083E0C0
:1014880012611174288E048F05FF1261018C598D29
:101498005AAE28AF29740A8E048F05FF1261018D98
:1014A800068C07AC59AD5ACFCECF120003740A8E02
:1014B800048F05FF1261018C598D5AAE28AF29128D
:1014C800615D8E288F29807DE564A859B800049550
:1014D8005A5072AE59AF5AE5641261558E598F5AF7
:1014E8007428BE00039F500C755A28755900740D56
:1014F800900047F0AE59AF5A900083E01261117422
:10150800288E048F05FF1261018C598D5AAE28AFC1
:1015180029740A8E048F05FF1261018D068C07ACB1
:1015280059AD5ACFCECF120003740A8E048F05FF2F
:101538001261018C598D5AAE28AF29EF2DFDEE3C72
:10154800FC8C288D29229000DEE0B4026AE55E75E5
:10155800F00884FF7E008F37E55E75F00884ADF0F3
:101568007C008D3A753F08755901755AE0E537C317
:10157800943F5005120B998006900277E0F5378565
:10158800372D752C00AE2CAF2DAC2AAD2B120003D5
:1015980074648E048F05FF1261018C2C8D2D9000D0
:1015A8007BE08C068D0712611174648E048F05FF31
:1015B8001261018C2C8D2DAE28AF29AC2AAD2B12CF
:1015C800000374648E048F05FF1261018C288D2935
:1015D80090007BE08C068D0712611174648E048F75
:1015E80005FF1261018C288D29A20D401DAE51AF57
:1015F800527405BE00039F5002D20DE560D394CC0F
:101608004008D2017411900047F09000DDE0B40268
:10161800089000DFE0640160028035AE28AF29E55C
:101628006A12611174E78E048F05FF1261018C281C
:101638008D299000DEE0B40217AE2CAF2DE56A12BA
:10164800611174E78E048F05FF1261018C2C8D2DBA
:1016580090009DE05402601B900094E0A851B800EF
:1016680012D39552400DA20DB3B35007E560C39451
:101678009A40028028AE35AF36900092E075F002AD
:10168800A4FDACF0EF2DFDEE3CFC74022DFD5001E5
:101698000CE560BC0007D39D4003754301856036A7
:1016A800753500E54370030217919000F0E0C3958B
:1016B800435003021783900100E0C394025076E57B
:1016C8006675F00A84FF7E00900578126138E0F5AF
:1016D8005A755900AE59AF5A900093E012611174CF
:1016E800648E048F05FF1261018C5B8D5C9000F0A5
:1016F800E004C395438C068D071261119000F0E059
:101708008E048F05FF1261018C5B8D5CAE28AF29BA
:10171800EF2DFDEE3CFC8C288D299000DEE0B40214
:1017280012AE2CAF2DAA5BAB5CEF2BFBEE3AFA8A1C
:101738002C8B2D80469000F0E004C39543854BF038
:10174800A4FFAEF09000F0E08E048F05FF12610157
:101758008C5B8D5CAE28AF29EF2DFDEE3CFC8C2810
:101768008D299000DEE0B40212AE2CAF2DAA5BAB3F
:101778005CEF2BFBEE3AFA8A2C8B2D05439000F098
:10178800E0C39543500375430090009DE054016009
:101798001B900091E0A851B80012D39552400DA2B9
:1017A8000DB3B35007E55EC394CC4002802590008A
:1017B8008FE075F003A4FFAEF0E5402FFF50010E57
:1017C80074032FFF50010EE55EBE0007D39F400350
:1017D800754401855E40E54470030218C49000F129
:1017E800E0C3954450030218B6900100E0C3940288
:1017F8005076E56675F00A84FF7E009005781261E0
:1018080038E0F55A755900AE59AF5A900090E01279
:10181800611174648E048F05FF1261018C5B8D5C0D
:101828009000F1E004C395448C068D071261119075
:1018380000F1E08E048F05FF1261018C5B8D5CAEB8
:1018480028AF29EF2DFDEE3CFC8C288D299000DE79
:10185800E0B40212AE2CAF2DAA5BAB5CEF2BFBEE13
:101868003AFA8A2C8B2D80469000F1E004C3954407
:10187800854CF0A4FFAEF09000F1E08E048F05FFD8
:101888001261018C5B8D5CAE28AF29EF2DFDEE3C1B
:10189800FC8C288D299000DEE0B40212AE2CAF2D0E
:1018A800AA5BAB5CEF2BFBEE3AFA8A2C8B2D054436
:1018B8009000F1E0C3954450037544009000F3E0B4
:1018C8002529FFAE2850010E8E288F299000A2E00E
:1018D800A828B80004952950099000A2E0F52975B8
:1018E80028009000DEE0B4020D9000A2E0A82CB819
:1018F8000006952D400280099000A2E0F52D752C78
:1019080000229000DEE0B401028003021A15A20D45
:10191800B35003021A139000A9E0B40168AE28AFCF
:1019280029AC51AD52120003743C8E048F05FF128E
:1019380061019000B9E0BC00109D400D9000BBE033
:10194800A828B8000495295002D202AE28AF29ACC5
:1019580051AD52120003743C8E048F05FF126101D1
:101968009000B9E0C3940ABC0015D39D40119000C3
:10197800BBE0C39405A828B80005D3952950028078
:1019880002C2028068AE28AF29AC51AD52120003E2
:1019980074788E048F05FF1261019000B9E0BC00D5
:1019A800109D400D9000BBE0A828B8000495295070
:1019B80004D2028038AE28AF29AC51AD52120003D0
:1019C80074788E048F05FF1261019000B9E0C3940A
:1019D8000ABC0015D39D40119000BBE0C39405A834
:1019E80028B80005D3952950028002C202A202B38A
:1019F8004019AE28AF299000BAE012611174648EC4
:101A0800048F05FF1261018C288D298002C202A271
:101A180000B34006A201B3B35009900015E4F0A347
:101A2800F08024AE28AF297400D39F74019E400C27
:101A3800900015E528F0A3E529F0800B74FF9000CD
:101A480015F8E4F0E8A3F09000C0E0D39402400C4D
:101A58009000ABE07006A20DB3B34002801AAE2826
:101A6800AF2974021261118E288F29AE2CAF2D7404
:101A7800021261118E2C8F2D9000A9E0B4011AAECC
:101A880028AF2974021261118E288F29AE2CAF2D30
:101A980074021261118E2C8F2DAE28AF29745E123C
:101AA8006111740A8E048F05FF1261018C288D293B
:101AB8009000DEE0B40217AE2CAF2D745E126111F7
:101AC800740A8E048F05FF1261018C2C8D2DAE28AF
:101AD800AF297402BE000AD39F40067529027528F3
:101AE80000AE2CAF2D7402BE000AD39F4006752DA0
:101AF80002752C00900013E528F0A3E529F0229048
:101B08000046E0900378126143E0F5417542649025
:101B18000046E0FE9000B4E0D39E4037E55E75F0E5
:101B28000884FF7E008F37E55E75F00884ADF07C91
:101B3800008D3A753F08755903755A96E537C39471
:101B48001F5005120B99800690042DE0F537853754
:101B5800428035E55E75F00884FF7E008F37E55ECC
:101B680075F00884ADF07C008D3A753F087559030F
:101B7800755AB6E537C3941F5005120B9980069025
:101B8800044DE0F537853742229000EAE0F53C75D0
:101B98003F11755904755A00AE51AF52E53C75F0C6
:101BA8000FA4FDACF0EDD39FEC9E4021E53C8E04E4
:101BB8008F05FF126101ED75F010A4FFAEF0E55E30
:101BC80075F01184FD7C00ED2FF53D800EE55E7506
:101BD800F01184FF7E00EF24F0F53D853D37E55E8A
:101BE80075F01184AFF07E008F3A120B9985373E5D
:101BF800AE51AF529000EAE075F00FA4FDACF0EDE5
:101C0800D39FEC9E4028755904755A10853D3712AC
:101C18000B99853E38853739AE51AF52E53C8E0475
:101C28008F05FF12612C8D3A853C3B120C138537CA
:101C380041754264229000EAE0F53C753F11755900
:101C480004755A00AE51AF52E53C75F00FA4FDACD7
:101C5800F0EDD39FEC9E4021E53C8E048F05FF12EA
:101C68006101ED75F010A4FFAEF0E56075F0118428
:101C7800FD7C00ED2FF53D800EE56075F01184FFC9
:101C88007E00EF24F0F53D853D37E56075F0118461
:101C9800AFF07E008F3A120B9985373EAE51AF52A6
:101CA8009000EAE075F00FA4FDACF0EDD39FEC9E38
:101CB8004028755904755A10853D37120B99853E91
:101CC80038853739AE51AF52E53C8E048F05FF1287
:101CD800612C8D3A853C3B120C1385374175426463
:101CE8009000E5E0B40479900046E0FE9000B4E08E
:101CF800D39E4037E55E75F00884FF7E008F37E598
:101D08005E75F00884ADF07C008D3A753F08755912
:101D180003755A96E537C3941F5005120B99800630
:101D280090042DE0F5378537428035E55E75F0087B
:101D380084FF7E008F37E55E75F00884ADF07C0087
:101D48008D3A753F08755903755AB6E537C3941F20
:101D58005005120B99800690044DE0F537853742FF
:101D68002290007EE0B4013BE56675F00A84FF7EB0
:101D7800008F37E56675F00A84ADF07C008D3A7502
:101D88003F0A755905755A12E537C3941150051263
:101D98000B99800690059BE0F537E5422537C394FB
:101DA80064F54290007FE0B4013BE56775F00A8472
:101DB800FF7E008F37E56775F00A84ADF07C008DF3
:101DC8003A753F0A755905755A7EE537C39411501F
:101DD80005120B998006900607E0F537E54225378E
:101DE800C39464F542E5412542F534900086E0B499
:101DF80002109007BEE02534FE9000DAE0F4042ECD
:101E0800F5349000DDE0D394014040E56AC394E7DF
:101E1800501D74E7C3956AFE9007C0E08E00F5F088
:101E2800E884FF7E008F37E5342537F534801CE5DC
:101E38006AC394E7FE9007C0E08E00F5F0E884FFDF
:101E48007E008F37E534C39537F534A20D4006E59B
:101E5800412464F534E534D394644009E534C394EB
:101E680064F53480037534009000B6E0C3953450AF
:101E7800069000B6E0F53422D200900070E0A85138
:101E8800B8000495525041900070E0A851B8000481
:101E98009552500375340F900070E004A851B800B3
:101EA800049552500375340A900070E02402A8513A
:101EB800B8000495525005753405C200900070E0D2
:101EC80060067409900047F0C23A7E017F009000D6
:101ED800BCE01261119000CBE08E048F05FF126107
:101EE80001E55EBC0017D39D40139000C5E0B40225
:101EF80004D23A8002C200740A900047F09000BDF4
:101F0800E0C3956650159000CFE0A851B80004953D
:101F1800525002C200740B900047F0E566C3946407
:101F2800501D900115E0600D900115E0A851B80012
:101F380006955240028008C200740B900047F0A238
:101F48000040037534059000FEE0B401149000FFD2
:101F5800E0A851B8000495525007E55EC3955F406C
:101F68000280089000A7E0F534803A900086E0B43B
:101F78000306A22AB3B34002802B9007C2E0C394A1
:101F880005A851B800049552500C9000A7E0F5340C
:101F9800740C900047F09007C2E0A851B80004956F
:101FA800525002C20085346B900078E02534FE90D0
:101FB8000046E075F01E84FC7F00EE2CF53422907C
:101FC8000046E075F00584FF7E008F37900046E0FC
:101FD80075F00584ADF07C008D3A753F05755903A1
:101FE800755AD69000C9E01475F00584FF7E00E5A7
:101FF80037BE00039F5005120B99800BE5379004FC
:102008004E126143E0F537E5379007C1F09007C1FC
:10201800E0FE9000B8E0C39E50089000B8E090073A
:10202800C1F022E56675F00A84FF7E0090057812FB
:102038006138E0F546E546D394644010E546C3941C
:102048006475F00F84FF7E008F468003754600900C
:10205800009BE02546F546229007B2E0FEA3E0FF8C
:102068007404120039E55E126111740F8E048F0535
:10207800FF1261019007B0ECF0A3EDF090008EE044
:10208800B40262E569C3944175F00584FF7E008F50
:1020980037E56975F00584ADF07C008D3A753F052C
:1020A800755906755A14E537C394175005120B99DC
:1020B800800690069FE0F5379007B0E0FEA3E0FFAA
:1020C800740A8E048F05FF126101E5378C068D07AF
:1020D800126111740A8E048F05FF1261019007B016
:1020E800ECF0A3EDF09007B0E0FEA3E0FF9007B698
:1020F800E0FCA3E0FDEDD39FEC9E400F9007B6E017
:10210800F8A3E09007B0C8F0A3C8F0229006BFE09B
:10211800903419F8282873804C85527280479000B3
:10212800CBE0855EF0A4FFAEF074081200398F7220
:102138008033856072802E856672802985677280FB
:1021480024856872801F856972801A856A72801575
:102158008565728010856472800B856B728006902D
:052168000016E0F57215
:1034190002211F02212102212602213A02213F0213
:10342900214402214902214E02215302215802213D
:073439005D02216202216720
:10216D009006C0E0FE9006C1E0D39E404B9006BFA6
:10217D00E0B404189006C1E0C395725002D22B90C2
:10218D0006C0E0D395724002C22B802A9006C0E0B3
:10219D00C3957250099006C1E0D39572500280022A
:1021AD00D22B9006C0E0D3957250099006C1E0C3C2
:1021BD0095725002C22B802A9006C0E0D3957240D2
:1021CD00099006C1E0C3957240028002C22B9006B1
:1021DD00C0E0C3957240099006C1E0D395724002EC
:1021ED00D22B229006C3E0903440F8282873804CFF
:1021FD0085527280479000CBE0855EF0A4FFAEF073
:10220D0074081200398F728033856072802E856656
:10221D007280298567728024856872801F85697236
:10222D00801A856A7280158565728010856472804A
:0C223D000B856B728006900016E0F572B5
:103440000221FB0221FD02220202221602221B029D
:10345000222002222502222A02222F0222340222C4
:073460003902223E02224363
:102249009006C4E0FE9006C5E0D39E405F9006C3A9
:10225900E0B404189006C5E0C395725002D22C90E0
:1022690006C4E0D395724002C22C803E9006C4E0B9
:10227900C3957250099006C5E0D395725002800249
:10228900D22C9006C4E0D3957250099006C5E0C3DC
:1022990095725002C22C9006C3E0B401099000D790
:1022A900E0D3956050028002C22C802A9006C4E0D7
:1022B900D3957240099006C5E0C395724002800229
:1022C900C22C9006C4E0C3957240099006C5E0D3BC
:1022D90095724002D22C229006C7E0903467F82804
:1022E9002873804C85527280479000CBE0855EF060
:1022F900A4FFAEF074081200398F728033856072C2
:10230900802E85667280298567728024856872802F
:102319001F856972801A856A7280158565728010B9
:10232900856472800B856B728006900016E0F572E9
:103467000222EB0222ED0222F202230602230B02C2
:10347700231002231502231A02231F0223240223E7
:073487002902232E0223336A
:102339009006C8E0FE9006C9E0D39E404B9006C7C0
:10234900E0B404189006C9E0C395725002D22D90EA
:1023590006C8E0D395724002C22D802A9006C8E0D3
:10236900C3957250099006C9E0D395725002800254
:10237900D22D9006C8E0D3957250099006C9E0C3E2
:1023890095725002C22D802A9006C8E0D3957240FA
:10239900099006C9E0C3957240028002C22D9006D9
:1023A900C8E0C3957240099006C9E0D3957240020E
:1023B900D22D229006CBE090348EF8282873804CD9
:1023C90085527280479000CBE0855EF0A4FFAEF0A5
:1023D90074081200398F728033856072802E856689
:1023E9007280298567728024856872801F85697269
:1023F900801A856A7280158565728010856472807D
:0C2409000B856B728006900016E0F572E7
:10348E000223C70223C90223CE0223E20223E7024C
:10349E0023EC0223F10223F60223FB022400022472
:0734AE000502240A02240FAD
:102415009006CCE0FE9006CDE0D39E404B9006CBD7
:10242500E0B404189006CDE0C395725002D22E9008
:1024350006CCE0D395724002C22E802A9006CCE0ED
:10244500C3957250099006CDE0D395725002800273
:10245500D22E9006CCE0D3957250099006CDE0C3FC
:1024650095725002C22E802A9006CCE0D395724018
:10247500099006CDE0C3957240028002C22E9006F7
:10248500CCE0C3957240099006CDE0D39572400229
:10249500D22E229006CFE09034B5F8282873804CD0
:1024A50085527280479000CBE0855EF0A4FFAEF0C8
:1024B50074081200398F728033856072802E8566AC
:1024C5007280298567728024856872801F8569728C
:1024D500801A856A728015856572801085647280A0
:0C24E5000B856B728006900016E0F5720B
:1034B5000224A30224A50224AA0224BE0224C302D4
:1034C50024C80224CD0224D20224D70224DC0224FB
:0734D500E10224E60224EBF2
:1024F1009006D0E0FE9006D1E0D39E404B9006CFEF
:10250100E0B404189006D1E0C395725002D22F9026
:1025110006D0E0D395724002C22F802A9006D0E007
:10252100C3957250099006D1E0D395725002800292
:10253100D22F9006D0E0D3957250099006D1E0C316
:1025410095725002C22F802A9006D0E0D395724036
:10255100099006D1E0C3957240028002C22F900615
:10256100D0E0C3957240099006D1E0D39572400244
:10257100D22F229006D3E09034DCF8282873804CC7
:1025810085527280479000CBE0855EF0A4FFAEF0EB
:1025910074081200398F728033856072802E8566CF
:1025A1007280298567728024856872801F856972AF
:1025B100801A856A728015856572801085647280C3
:0C25C1000B856B728006900016E0F5722E
:1034DC0002257F02258102258602259A02259F025C
:1034EC0025A40225A90225AE0225B30225B8022582
:0734FC00BD0225C20225C735
:1025CD009006D4E0FE9006D5E0D39E404B9006D306
:1025DD00E0B404189006D5E0C395725002D2309045
:1025ED0006D4E0D395724002C230802A9006D4E022
:1025FD00C3957250099006D5E0D3957250028002B2
:10260D00D2309006D4E0D3957250099006D5E0C330
:10261D0095725002C230802A9006D4E0D395724054
:10262D00099006D5E0C3957240028002C230900633
:10263D00D4E0C3957240099006D5E0D3957240025F
:10264D00D230229006D7E0903503F8282873804CBD
:10265D0085527280479000CBE0855EF0A4FFAEF00E
:10266D0074081200398F728033856072802E8566F2
:10267D007280298567728024856872801F856972D2
:10268D00801A856A728015856572801085647280E6
:0C269D000B856B728006900016E0F57251
:1035030002265B02265D02266202267602267B02E3
:10351300268002268502268A02268F022694022608
:073523009902269E0226A377
:1026A9009006D8E0FE9006D9E0D39E404B9006D71D
:1026B900E0B404189006D9E0C395725002D2319063
:1026C90006D8E0D395724002C231802A9006D8E03C
:1026D900C3957250099006D9E0D3957250028002D1
:1026E900D2319006D8E0D3957250099006D9E0C34B
:1026F90095725002C231802A9006D8E0D395724073
:10270900099006D9E0C3957240028002C231900651
:10271900D8E0C3957240099006D9E0D3957240027A
:10272900D231229006DBE090352AF8282873804CB4
:1027390085527280479000CBE0855EF0A4FFAEF031
:1027490074081200398F728033856072802E856615
:102759007280298567728024856872801F856972F5
:10276900801A856A72801585657280108564728009
:0C2779000B856B728006900016E0F57274
:10352A0002273702273902273E022752022757026B
:10353A00275C02276102276602276B02277002278F
:07354A007502277A02277FBA
:102785009006DCE0FE9006DDE0D39E404B9006DB34
:10279500E0B404189006DDE0C395725002D2329081
:1027A50006DCE0D395724002C232802A9006DCE056
:1027B500C3957250099006DDE0D3957250028002F0
:1027C500D2329006DCE0D3957250099006DDE0C365
:1027D50095725002C232802A9006DCE0D395724091
:1027E500099006DDE0C3957240028002C232900670
:1027F500DCE0C3957240099006DDE0D39572400296
:10280500D232229006DFE0903551F8282873804CAB
:1028150085527280479000CBE0855EF0A4FFAEF054
:1028250074081200398F728033856072802E856638
:102835007280298567728024856872801F85697218
:10284500801A856A7280158565728010856472802C
:0C2855000B856B728006900016E0F57297
:1035510002281302281502281A02282E02283302F3
:10356100283802283D02284202284702284C022816
:073571005102285602285BFD
:102861009006E0E0FE9006E1E0D39E404B9006DF4B
:10287100E0B404189006E1E0C395725002D233909F
:1028810006E0E0D395724002C233802A9006E0E070
:10289100C3957250099006E1E0D39572500280020F
:1028A100D2339006E0E0D3957250099006E1E0C37F
:1028B10095725002C233802A9006E0E0D3957240AF
:1028C100099006E1E0C3957240028002C23390068E
:1028D100E0E0C3957240099006E1E0D395724002B1
:1028E100D233229006E3E0903578F8282873804CA3
:1028F10085527280479000CBE0855EF0A4FFAEF078
:1029010074081200398F728033856072802E85665B
:102911007280298567728024856872801F8569723B
:10292100801A856A7280158565728010856472804F
:0C2931000B856B728006900016E0F572BA
:103578000228EF0228F10228F602290A02290F027E
:10358800291402291902291E02292302292802299D
:073598002D02293202293740
:10293D009006E4E0FE9006E5E0D39E404B9006E362
:10294D00E0B404189006E5E0C395725002D23490BD
:10295D0006E4E0D395724002C234802A9006E4E08A
:10296D00C3957250099006E5E0D39572500280022E
:10297D00D2349006E4E0D3957250099006E5E0C399
:10298D0095725002C234802A9006E4E0D3957240CD
:10299D00099006E5E0C3957240028002C2349006AC
:1029AD00E4E0C3957240099006E5E0D395724002CC
:1029BD00D23422AE2EAF2F74F5D39F74019E4008F2
:1029CD00782E126165022ADA752F01752E00AE512F
:1029DD00AF52E546BE000DD39F40099000ADE0D348
:1029ED00954740028023754700E546C39552F57221
:1029FD009000B0E0D395454008E5452572F545803A
:102A0D00069000B0E0F54580020547900089E0D3BF
:102A1D009560401CE55EC3955F4015AE51AF52E524
:102A2D0046BE00039F50099000AEE0D3954840028A
:102A3D00806E9007C5E0A851B800049552500375FB
:102A4D004A009007C5E0A851B8000BD39552400637
:102A5D00E5529007C5F0E54A7041E552C39546F53C
:102A6D0072E572D3940540037572059000AFE0C313
:102A7D0095455007E572C3954540028009E545C36C
:102A8D009572F54580069000AFE0F5459000AFE0FA
:102A9D00D3954540069000AFE0F54575480080029E
:102AAD000548E54A7016900089E0C39560500DE524
:102ABD00462405A851B8000695524002800F90009B
:102ACD009CE0F545754A0174789007C5F022AE2E4D
:102ADD00AF2F74E9D39F74039E4008782E12616561
:102AED00022C79752F01752E00754532A235402ABD
:102AFD0075451990009CE075F002A4FFAEF0E54716
:102B0D00BE0006D39F4002D2350547754A0374783F
:102B1D009007C5F0754900022C68AE51AF52E546DD
:102B2D006F4E7003022C68E546BE000DD39F400921
:102B3D009000ADE0D395474002800F754700E54A00
:102B4D00C394035003754519800DE546C39552F5A1
:102B5D0072E5472572F547900089E0D39560400EE8
:102B6D009007C5E0A851B80007D395524002800CDC
:102B7D00054990009CE0B54903754A00E54AB40348
:102B8D0006A20DB3B34002800A0549E549B43C03E2
:102B9D00754A02E54AB402299007C5E0A851B8006C
:102BAD000ED395524009E5529007C5F07549009036
:102BBD000089E0C39560500975490074789007C588
:102BCD00F0E54A705A900089E0D39560401CE55EAF
:102BDD00C3955F4015AE51AF52E546BE00039F5001
:102BED00099000AEE0D39548400280087548007505
:102BFD00454B8028E552C39546F572E572D3940591
:102C0D004003757205900089E0D395604008E54852
:102C1D002572F5488006E5482406F548754900E516
:102C2D004A7016900089E0C39560500DE546240565
:102C3D00A851B80006955240028003754A01E54A35
:102C4D00B40118754519054990009CE0B549067504
:102C5D004A0275490074789007C5F0E54575F00A8C
:102C6D00A4FFAEF09007BAEEF0A3EFF022E56E9060
:102C7D00359FF8282873900081E07003022E28906C
:102C8D0000B7E0B401028003022D78900044E0B556
:102C9D005D028003022D757E017F00E5BE1261117C
:102CAD00E5BD2FFF50010E8E598F5A741012611110
:102CBD0090006FE08E048F05FF1261019007C6EC46
:102CCD00F0A3EDF0E56A60089000DDE064026002BB
:102CDD0080269000DFE0B4011F9007C6E0FEA3E060
:102CED00FF74E7126111E56A8E048F05FF12610111
:102CFD009007C6ECF0A3EDF0900081E0B4022790B0
:102D0D0007C8E0FEA3E0FF9007C6E0FCA3E0FDEFDF
:102D1D002DFDEE3CFC74018C068D071200399007D9
:102D2D00C6EEF0A3EFF09007C6E0FEA3E0FF90071C
:102D3D00C8E0FCA3E0FDEDD39FEC9E4004D23880AB
:102D4D0002B2389007C6E0F8A3E09007C8C8F0A318
:102D5D00C8F09000B3E064016006A238B3B340023E
:102D6D0080069007C7E0F55E022E26D2387E017FE1
:102D7D0000E5BE126111E5BD2FFF50010E8E598F7A
:102D8D005A741012611190006FE08E048F05FF12BE
:102D9D0061019007C6ECF0A3EDF0E56A60089000C4
:102DAD00DDE06402600280269000DFE0B4011F9038
:102DBD0007C6E0FEA3E0FF74E7126111E56A8E0419
:102DCD008F05FF1261019007C6ECF0A3EDF09000A6
:102DDD0081E0B402279007C8E0FEA3E0FF9007C68C
:102DED00E0FCA3E0FDEF2DFDEE3CFC74018C068DA7
:102DFD00071200399007C6EEF0A3EFF09007C6E07A
:102E0D00F8A3E09007C8C8F0A3C8F09000B3E06441
:102E1D000160069007C7E0F55E8003755E009000C7
:102E2D007DE07006756E01022C7A75BB180233F3C6
:102E3D0090007DE07003022FC97E017F00E5BE1278
:102E4D006111E5BD2FFF50010E8E598F5A9000C3B1
:102E5D00E0B4010F7E0F7FFFAC59AD5A12615D8E4C
:102E6D00598F5A9000E8E0B40245AE59AF5A900020
:102E7D001FE0FCA3E0FDEDD39FEC9E400A90001FE8
:102E8D00E559F0A3E55AF0AE59AF5A900021E0FC98
:102E9D00A3E0FDEFD39DEE9C400A900021E559F093
:102EAD00A3E55AF0AE59AF5A74041200398F6090F1
:102EBD0000E8E0704CAE59AF5A90001FE0FCA3E063
:102ECD00FDEFD39DEE9C400912615D8E598F5A80A6
:102EDD0006755A00755900AE59AF5A74101261112A
:102EED0090006CE08E048F05FF1261018C598D5A94
:102EFD0074FFBC0009D39D4005855A608003756041
:102F0D00FE9000B3E0B401028003022FC7A20DB3FF
:102F1D00B3500E900087E0A851B80005D3955250DC
:102F2D0003022FBC900088E075F019A4FFAEF0905D
:102F3D0000CBE08E048F05FF1261019000C4E08587
:102F4D0060F0A4FFAEF074648D028C038E048F05C7
:102F5D00FF126101EA2DFDEB3CFC8C598D5AE56A9F
:102F6D00600F9000DDE0B402089000DFE0640160C6
:102F7D00028017AE59AF5A74E7126111E56A8E04DB
:102F8D008F05FF1261018C598D5AAE59AF5A9007BA
:102F9D00C6E0FCA3E0FDEDD39FEC9E4005855A5E97
:102FAD00800BA238B340069007C7E0F55E800BA2F8
:102FBD0038B340069007C7E0F55E8003756000905A
:102FCD000080E07006756E02022C7A75BB19023313
:102FDD00F3900080E0700302307EE55DD3955040A4
:102FED000302307C90001DE0FEA3E0FFE56412615A
:102FFD005590001DEEF0A3EFF07E017F00E5BE12AF
:10300D006111E5BD2FFF50010E8E598F5A9000EDC5
:10301D00E07013740A12611174518E048F05FF1242
:10302D0061018D648019AE59AF5A740A1261118F06
:10303D00048E057E017F95CDCCCD125FFF8F64E5AB
:10304D0064D39464400375646490001DE0FEA3E0B6
:10305D00FFE5642FFF50010E90001DEEF0A3EFF081
:10306D00900084E0048E048F05FF1261018D648051
:10307D00037564329000D0E07006756E03022C7AF1
:10308D0075BB130233F39000D0E0604A7E017F00E0
:10309D00E5BE126111E5BD2FFF50010E8E598F5AFD
:1030AD0074041200398F659000D2E08565F0A4FD9F
:1030BD00ACF07464FF1261018D659000D1E08565FF
:1030CD00F0A4FFAEF074FF8E048F05FF126101EDC9
:1030DD0090006BF0800375650090007EE0700675C2
:1030ED006E04022C7A75BB170233F390007EE0B4A8
:1030FD000102800302318C7E017F00E5BE12611159
:10310D00E5BD2FFF50010E8E598F5A9007CAE06012
:10311D00199007CAE014905B9112008CE493FC7433
:10312D000193FDEDC39FEC9E400280069007CAE01F
:10313D0014F09007CAE0C394B3501DAE59AF5A9026
:10314D0007CAE004905B9112008CE493FC74019328
:10315D00FDEFC39DEE9C400280069007CAE004F08F
:10316D009007CAE0FE9000A4E08E0088F0A4FFAEA8
:10317D00F074648E048F05FF1261018D66800375F6
:10318D00660090007FE07006756E05022C7A75BBA7
:10319D00160233F390007FE0B40102800302323552
:1031AD007E017F00E5BE126111E5BD2FFF50010EBE
:1031BD008E598F5A9007CBE060199007CBE0149091
:1031CD005CFB12008CE493FC740193FDEDC39FEC4A
:1031DD009E400280069007CBE014F09007CBE0C331
:1031ED0094B3501DAE59AF5A9007CBE004905CFBE1
:1031FD0012008CE493FC740193FDEFC39DEE9C4093
:10320D000280069007CBE004F09007CBE0FE900023
:10321D00AAE08E0088F0A4FFAEF074648E048F05D2
:10322D00FF1261018D67800375670075BB1F023347
:10323D00F37E017F00E5BE126111E5BD2FFF500148
:10324D000E8E598F5A740912611174E68E048F0512
:10325D00FF1261018D69900086E07006756E0702A0
:10326D002C7A75BB150233F3900086E070030233A0
:10327D008F7E017F00E5BE126111E5BD2FFF50016C
:10328D000E8E598F5A74041200398F68900086E0A3
:10329D00B401159000DAE08568F0A4FFAEF0740774
:1032AD00120039EF9007BFF0900086E0B402159040
:1032BD0000DAE08568F0A4FFAEF07407120039EF74
:1032CD009007BEF0900086E0B40302800302338DB8
:1032DD009000C7E070389000DAE0601CE568C39498
:1032ED00195002D22AE568D394644002C22A900094
:1032FD00A6E09007C2F08014E568C394195002D27D
:10330D0039E568D394324002C239C22A80639000F5
:10331D00A6E070349000DAE08568F0A4FFAEF0749A
:10332D00FF8E048F05FF126101ED9007C2F0AE51C3
:10333D00AF52741EBE0006D39F4002D22AE560D361
:10334D0094E54002C22A8029E568C3940A500DAE67
:10335D0051AF52741EBE0004D39F50028002D22A78
:10336D00E560D394E54002C22A9000A6E09007C222
:10337D00F09007C2E0C39405500674059007C2F0A3
:10338D0080037568009000DDE07006756E08022CF4
:10339D007A75BB1480509000DDE060397E017F00AE
:1033AD00E5BE126111E5BD2FFF50010E8E598F5AEA
:1033BD00EFD39421EE940E4005756AFF8015AE593A
:1033CD00AF5A741012611174E38E048F05FF1261F0
:1033DD00018D6A8003756A00900081E0600575BB00
:0633ED001A800375BB18F5
:10359F00022C83022E3D022FDE0230930230F802FE
:0B35AF0031A102323E0232750233A34C
:0533F300056ED2EC2282
:096143002582F582500205832239
:0F008C0025E050020583258250020583F582226C
:1060E000EF2F500205832582F582E5833E2EF5834E
:0160F000228D
:10615500CFC39FFF50011E22C3EF9DFFEE9CFE2281
:086165000806B600021806222C
:0D611F00A3E004F07006120049E004F02235
:0E003900048007C3CE13CECF13CFD5E0F6223E
:105FFF00BC000FBE0008ED8FF084FFADF022E4FE71
:10600F00FF22BE000DEF60FE54F0606F20E7030229
:10601F0060B5EAC0E0EBC0E078017A0075F001EE00
:10602F0020E710EF25E0FFEE33FE0AC5F023C5F0A1
:10603F0030E7F0EA5407F9096A7A007B006001083B
:10604F00C3EC9E40167004ED9F4010ED9FFDEC9E3B
:10605F00FCE5F0CA4ACA03F5F08005E5F003F5F058
:10606F00C3EE13FEEF13FFD9D77908CACBCAD8D026
:10607F00EAFEEBFFD0E0FBD0E0FA22EC8FF084FCDD
:10608F00ED54F045F0C48FF084FEEDC454F045F0AC
:10609F00C48FF084FDEEC4FE54F02DFFEE540F3C80
:1060AF00FEADF07C0022790078008FF0EC7E0820A6
:1060BF00E70DC3CD33CD33C933C9C833C8DEF08440
:1060CF0049F9E5F08FF0BE00E6FD7C00E9FFE8FE40
:0160DF00229E
:0E611100F88FF0A4FFE5F0CE88F0A42EFE2259
:10000300EF8DF0A4F9A8F0EF8CF0A428F8EE8DF0B2
:06001300A428FEE9FF2213
:1060F100600D782B0260FB007830D8FED5E0F822E5
:10610100EEC0E07E00125FFFEFFDEEFCD0E0FE226C
:0C612C00EEC0E07E00125FFFD0E0FE221B
:03001B0002001EC2
:0300530002005652
:03009B00020071EF
:0300000002614C4E
:09614C0075817475D000023EA7B4
:0B613800E5822FF582E5833EF583220F
:0A0049000582D5820215831582227C
:10001E00C0E0C0F0C083C082C0D075D000123DD900
:0B002E00D0D0D082D083D0F0D0E032E0
:10005600C0E0C0F0C083C082C0D075D000123DDCC5
:10006600D0D0D082D083D0F0D0E032C0E0C0F0C093
:1000760083C082C0D075D000123E5AD0D0D082D074
:0600860083D0F0D0E0324F
:00000001FF
